:1000000000008A150A16882E0528831606309F00E0
:1000100085018601F0308700FF308800FF309200B4
:100020008312FF3092000F309700171297121D12A3
:100030009D120F309D000130A0001C30A10007145C
:10004000871596309B0047309500A0309B00081E16
:100050002C2808192C283220081D2528081A2528A4
:100060003D20252846309B005E20230895009920DE
:10007000081D3228081E3228080046309B00482000
:10008000230895009920081D3D28081E3D280800DA
:10009000A1030319A003211C171221181716A11C74
:1000A0009712A11897162008A2002108A300031098
:1000B000A20CA30C0310A20CA30C0800A10A0319A4
:1000C000A00A211C171221181716A11C9712A1189B
:1000D00097162008A2002108A3000310A20CA30C6D
:1000E0000310A20CA30C0800000000000000000098
:1000F0000000000008000000A43087280000403005
:1001000087281F30872800000E3087280530A4007C
:10011000A40B88280800C8309A2864309A28323006
:100120009A2814309A280A309A2805309A280230E2
:100130009A280130A500F930A4000000A40B9D28E6
:10014000A50B9B280800C830AE286430AE2832309A
:10015000AE281430AE280A30AE280530A600643030
:10016000A500F930A4000000A40BB328A50BB1280A
:10017000A60BAF280800BD280530A5006430A400F8
:10018000F930A3000000A30BC228A40BC028A50BC4
:10019000BE280800A50BC12808004E08033C031D1B
:1001A000D5284C088400013080005014DB285018FA
:1001B000CF0ACE015010CD0ABC285018CF0A4F08E4
:1001C000F80000345008F8014F020318EA284F08DD
:1001D000F700F628F7010830D100CF0DF70D5008D1
:1001E00077020318F700F80DD10BED2800347808DA
:1001F0004D08CF006430D000E2207708CD007808A9
:100200003030031D0A294E181129CE1911294E1A12
:1002100020300C29CE114E12F80778080C1E0E293A
:1002200099004D08CF000A30D000E2207708CD00B9
:1002300078083030031D2029CE1925294E1A203088
:10024000F80778080C1E222999003030CD074D0898
:100250000C1E282999008A110A125E2CF701F80158
:100260004B0803104C18F707F70CF80CCC18F707DD
:10027000F70CF80C4C19F707F70CF80CCC19F7072A
:10028000F70CF80C4C1AF707F70CF80CCC1AF70718
:10029000F70CF80C4C1BF707F70CF80CCC1BF70706
:1002A000F70CF80C8A110A12812C43148D11941347
:1002B0008316111483128D195629941B56298316FF
:1002C000111C642983125F29A1308312C5003328D1
:1002D0000130F70045207808A9000130F7004520DB
:1002E0007808AA000130F70045207808AB000130FB
:1002F000F70045207808AC000130F7004520AE013A
:100300007808AD00F70145200030AD070318AE0AAC
:100310007808AE078316111511198C298312C701AD
:100320002908C500290831020319982900309929A4
:100330000130C9002908B100C9080319AA290A30E7
:100340000C1EA02999000D300C1EA4299900450807
:10035000CB0054204508CB004730CC00B5207808AE
:10036000C600460B042AC7080319042A0A30CB002A
:1003700041300C1EB9299900CB0BB829AF18C229FE
:100380000130AF06AF1400302F180130003A031DC2
:10039000E7290730CA004508F7004A08F8000319A2
:1003A000D5290310F70CF80BD129771CD929CA03DA
:1003B000CB290130F7004A08F8000319E32903109C
:1003C000F70DF80BDF297708FF3AC505032ACA01A4
:1003D0004508F7004A08F8000319F2290310F70C42
:1003E000F80BEE29771CF629CA0AE8290130F70034
:1003F0004A08F8000319002A0310F70DF80BFC292E
:100400007708FF3AC505EA2A460832020318962AF9
:100410001230CB0042300C1E0B2A9900CB0B0A2A5B
:10042000AF184A2AC5080319172A0030182A0130C4
:100430003005CC003008CD004C08CE00CF014F086D
:10044000073C031C432A4D08F7004F08F800031926
:100450002D2A0310F70CF80B292A771C322A0030BA
:10046000F800452A4E08F7004F08F80003193C2A07
:100470000310F70CF80B382A771C412A0130F800DA
:10048000452ACF0A1F2A0130F8007818492A2F1070
:100490004A2A2F14AF104508CB004830CC00B520B5
:1004A0007808013C0318952A00302F180130013CD0
:1004B000031D782A0730CA004508F7004A08F800EB
:1004C0000319662A0310F70CF80B622A77186A2AB8
:1004D000CA035C2A0130F7004A08F8000319742A9D
:1004E0000310F70DF80B702A7708FF3AC505942A18
:1004F000CA014508F7004A08F8000319832A0310C7
:10050000F70CF80B7F2A7718872ACA0A792A013054
:10051000F7004A08F8000319912A0310F70DF80BA9
:100520008D2A7708FF3AC5054B2AEA2A1130CB00FD
:1005300043300C1E992A9900CB0B982A4508CB0012
:100540004830CC00B5207808013C0318EA2AF701AE
:10055000AF1877142F08770601390319CD2A073011
:10056000CA004508F7004A08F8000319BB2A03101F
:10057000F70CF80BB72A7718BF2ACA03B12A013043
:10058000F7004A08F8000319C92A0310F70DF80B01
:10059000C52A7708FF3AC505E92ACA014508F700C8
:1005A0004A08F8000319D82A0310F70CF80BD42ACC
:1005B0007718DC2ACA0ACE2A0130F7004A08F80068
:1005C0000319E62A0310F70DF80BE22A7708FF3A21
:1005D000C5059E2A4608B2004508B00000302F1815
:1005E0000130CB004508CC004B08CD00CE01CF0137
:1005F0004F08073C031C0A2B4C08F7004F08F80073
:100600000319062B0310F70CF80B022B7718CE0AF0
:10061000CF0AF82A4E08023C0318542B4D0B322BFC
:10062000CF014E08023C0318312B4C08F7004F084D
:10063000F80003191F2B0310F70CF80B1B2B771C6A
:100640002F2B0130F7004F08F80003192B2B031054
:10065000F70DF80B272B7708FF3ACC05CE03CF0A0E
:10066000112B542B0730CF004E08023C0318542B9B
:100670004C08F7004F08F8000319422B0310F70C41
:10068000F80B3E2B771C522B0130F7004F08F80077
:1006900003194E2B0310F70DF80B4A2B7708FF3A7E
:1006A000CC05CE03CF03342B4C08F8007808C500E6
:1006B0004508803A03198A2B403A03198F2B803A58
:1006C0000319942B203A0319992B403A03199E2BB6
:1006D000103A0319A32B203A0319A82B083A03193F
:1006E000AC2B103A0319AF2B043A0319B32B083A79
:1006F0000319B72B023A0319BB2B043A0319BF2B7A
:10070000013A0319C32B023A0319C72B013A031903
:10071000CB2BDF2BFF30B600F930B500082CFF30B3
:10072000B600FA30B500082CFF30B600FB30B5003B
:10073000082CFF30B600FC30B500082CFF30B600A6
:10074000FD30B500082CFF30B600FE30B500082C97
:10075000FF30B600B500082CB601B501082CB60173
:100760000130B500082CB6010230B500082CB601E6
:100770000330B500082CB6010430B500082CB601D2
:100780000530B500082CB6010630B500082CB601BE
:100790000730B500082CB61BD82BB608031DD42B88
:1007A0003508003C0318D82BB6010830B500DE2B05
:1007B000B61FDE2BFF30B600F830B500082C450818
:1007C000CB00CC01CB1BCC034B1BCC03CB1ACC03F3
:1007D0004B1ACC03CB19CC0A4B19CC0ACB18CC0A38
:1007E0004B18CC0ACC1BFB2B4C08003C0318FB2BF2
:1007F000FA010130FC2B0030F800F8080319042C32
:10080000B6010430B500082CFF30B600FC30B5004E
:1008100037083502F7003608FA003808031C380F8D
:10082000FA0277083507F8000318FA0A3608FA07BB
:100830007808B9070318BA0A7A08BA073608B80060
:100840003508B700BA1B342C3A08003C0318342C86
:10085000FF3A031D2F2C3908873C0318342C013034
:10086000BA008730B900402CBA1B3D2CBA08031DD2
:10087000402C3908AC3C031C402CBA01AD30B90007
:10088000C9080319622C4508CB00542000302F18EA
:100890000130013C031D4F2CFA014930502C4430EB
:1008A000CC004C080C1E522C990020300C1E562CEB
:1008B00099003908CD001830CE00F72820300C1EE2
:1008C0005F2C99003A08F9003908F800F90CF80C87
:1008D000F90CF80CF90C78089500F90C790C303902
:1008E000F7001708CF39770497001030C5002A08A1
:1008F0004502C8003D082A02CA00CB000330CC00E4
:100900002E2978084807FA01F700F71BFA03C600FA
:100910007A08C70045082A020318A92C46083B0795
:10092000C8003C08C9000318C90A4708C907C91B01
:10093000A22C4908033C0318A22C0330BC00FF3052
:10094000BB00A82C4608BB070318BC0A4708BC0715
:10095000D32C2A0845020318D32C003083168800B4
:10096000FF308312880046083B02C8003C08C900DB
:100970004708031C470FC902C91BC82C4908013C82
:10098000031CCD2C031DC82C48082B3C031CCD2C6C
:100990000130BC002C30BB00D32C4608BB024708FA
:1009A000031C470FBC02FF309B002A08BD000B113F
:1009B0008A110A121D284230840000080319EF2C06
:1009C0000130F800F701F70BE32CF80BE22C4A306A
:1009D000F700F70BE92C00000000800BE02C8A11D7
:1009E0000A12852D28112808831687008312071103
:1009F0000C309700A81028088316870083128710F0
:100A00000C309D0095019B018A110A12962D071446
:100A1000281028088316870083128A110A12972D3E
:100A20001F3083055030F700203084008001840A95
:100A3000F70B162DF101F201F301F401F501F601B6
:100A4000F801F901FA01FB01FC01FD01FE01503042
:100A5000F700A03084008001840AF70B2B2DA00141
:100A600084011F30830583161F149F141F159F11C7
:100A7000073083129F000C308316990026309800AF
:100A8000903083129800A8152808831687008312D7
:100A90002816280883168700013093002830831217
:100AA0009400831694131413FF308312A800A90135
:100AB000AA01AB01AC01AD01AE012F14AF10B00122
:100AC000B101B201B301B401B501B601B701B8017A
:100AD0001A30B9000130BA00BB01BC01BD01BE0132
:100AE000BF01C001C1010D300C1E742D9900C10160
:100AF00041084F3C031C822D0A300C1E7D2D9900AD
:100B0000C10A782DFA30C200DB2C7830F8000638A4
:100B10009200FF3083169200831290018316010821
:100B2000C0390838810083128B16F22C072DC03093
:100B30008B04992D9A2D8B16F92C0E2DC0308B0419
:100B4000A02DA12DAE012F14AF10B001B101B20143
:100B5000B301B401B501B601B701B8011A30B9004B
:100B60000130BA00BB01BC01BD01BE01BF01C00123
:100B7000C1010D300C1EBA2D9900C10141084F3C36
:100B8000031CC82D0A300C1EC32D9900C10ABE2DAE
:100B9000FA30C200212D7830F80006389200FF307C
:100BA000831692008312900183160108C039083819
:100BB000810083128B16382D4D2DC0308B04DF2D14
:100BC000E02DC81BED2D4808013C031CF22D031D30
:100BD000ED2D47082B3C031CF22D0130BC002C30BE
:100BE000BB00F82D4508BB024608031C460FBC029B
:100BF000FF309B002A08BD00C70147084820C70AEC
:100C0000F70077080C1E022E990004304702031DDE
:100C1000FD2D103084003C08C9003B08C800442A60
:100C200009300C1E112E990020300C1E152E990033
:100C300020300C1E192E99000B118A110A121D2842
:100C40004130840000080319342E0130F800F70108
:100C5000F70B282EF80B272E4A30F700F70B2E2E15
:100C600000000000800B252E8A110A12BA2E2811CE
:100C7000280883168700831207110C309700A810EC
:100C8000280883168700831287100C309D00950179
:100C90009B018A110A12CB2E0714281028088316EC
:100CA000870083128A110A12CC2E1F308305503020
:100CB000F700203084008001840AF70B5B2EF101DD
:100CC000F201F301F401F501F601F801F901FA016D
:100CD000FB01FC01FD01FE015030F700A030840053
:100CE0008001840AF70B702EA00184011F30830558
:100CF00083161F149F141F159F11073083129F0026
:100D00000C3083169900263098009030831298009A
:100D1000A81528088316870083122816280883162A
:100D200087000130930028308312940083169413B7
:100D30001413FF308312A800A901AA01AB01AC0172
:100D4000AD01AE012F14AF10B001B101B201B3017A
:100D5000B401B501B601B701B8011A30B9000130CC
:100D6000BA00BB01BC01BD01BE01BF01C001FA3028
:100D7000C100202E7830F80006389200FF3083162C
:100D800092008312900183160108C039083881004F
:100D900083128B16372E4C2EC0308B04CE2ECF2EC6
:100DA0007830F80006389200FF30831692008312E4
:100DB000900183160108C0390838810083128B1610
:100DC0004D2E622EC0308B04E42EE52E4402031D0E
:100DD000DD2E3B08CA003A08C9003908C8003808A7
:100DE000C700CE01CD010130CC000630CB00D021B0
:100DF0000830C50045086620C50AF70077080C1EB4
:100E0000FF2E99000C304502031DFA2E2B08C80056
:100E10001830C9008D240E30C60046086620C60A68
:100E2000F70077080C1E122F990017304602031D99
:100E30000D2F4308CA004208C9004108C8004008F5
:100E4000C700CE01CD010130CC000630CB00D0214F
:100E50001930C70047086620C70AF70077080C1E3C
:100E60002F2F99001D304702031D2A2F2C08C80080
:100E70001830C9008D2455300C1E3C2F99000714E2
:100E800028102808831687008312071028102808C6
:100E900083168700C8308312B400D62C6E2D4F2FD6
:100EA0000330AE002E300C1E532F9900AE0B522F84
:100EB0000A300C1E592F99000D300C1E5D2F990021
:100EC000AD012D08F422AD0AF70077080C1E662F3D
:100ED000990029302D02031D612F0A300C1E6E2F40
:100EE00099000D300C1E722F9900AD012D0825239D
:100EF000AD0AF70077080C1E7B2F990014302D02E5
:100F0000031D762F83160C148C148C15C03083129D
:100F10008B048B168A2F8B2FB301B4011A30B500C6
:100F20000130B600B701B801B901BA01BB01BC017B
:100F30007830F80006389200FF3083169200831252
:100F4000900183160108C03903388100FA308312FA
:100F5000BD00052F8B161C2FC0308B040B30BD003D
:100F60002D300C1EB12F9900BD0BB02FBE013E08D5
:100F70003B21BE0AF70077080C1EBC2F99001C30DD
:100F80003E02031DB72F0F30BF002D300C1EC62FA1
:100F90009900BF0BC52F0630C0000A300C1ECE2FA3
:100FA0009900C00BCD2F0D300C1ED42F9900312F7E
:100FB000D82FD92FFF3FFF3FFF3FFF3FFF3FFF3FAE
:100FC000FF3FFF3FFF3FFF3FFF3FFF3FFF3FFF3F31
:100FD000FF3FFF3FFF3FFF3FFF3FFF3FFF3FFF3F21
:100FE000FF3FFF3FFF3FFF3FFF3FFF3FFF3FFF3F11
:100FF000FF3FFF3FFF3FFF3FFF3FFF3FFF3FFF3F01
:101000001F3083055030F700203084008001840AAF
:10101000F70B0628F101F201F301F401F501F601E5
:10102000F801F901FA01FB01FC01FD01FE0150305C
:10103000F700A03084008001840AF70B1B28A00170
:1010400084011F30830583161F149F141F159F11E1
:10105000073083129F000C308316990026309800C9
:10106000903083129800A8152808831687008312F1
:101070002816280883168700013093002830831231
:101080009400831694131413FF308312A800A9014F
:10109000AA01AB01AC01AD01AE012F14AF14B00138
:1010A000B101B201B301B4011A30B5000130B6008C
:1010B000B701B801B901BA01BB01BC017830F80031
:1010C00006389200FF308316920083129001831637
:1010D0000108C03903388100FA308312BD008A113B
:1010E0005B2F8A158B168A11722F8A15C0308B04DC
:1010F0000B30BD002D300C1E7B289900BD0B7A28CB
:10110000BE013E088A113B218A15BE0AF700770806
:101110000C1E882899001C303E02031D81280F30C8
:10112000BF002D300C1E92289900BF0B912806306D
:10113000C0000A300C1E9A289900C00B99280D3067
:101140000C1EA02899008A11872F8A15A628A72887
:10115000FF3FFF3FFF3FFF3FFF3FFF3FFF3FFF3F9F
:10116000FF3FFF3FFF3FFF3FFF3FFF3FFF3FFF3F8F
:10117000FF3FFF3FFF3FFF3FFF3FFF3FFF3FFF3F7F
:10118000FF3FFF3FFF3FFF3FFF3FFF3FFF3FFF3F6F
:103D00008A150A16802E8A01000000308A00102DC4
:103D1000031E832E903098008316181598161930BC
:103D2000990083120330FA00313090000C14EC2615
:103D3000EA3A031DAF2EFA01B62EEC26F900E33A5B
:103D40000319B82E7908EA3A0319B62E7908ED3A24
:103D5000031D9D2EE430E7260330FA00EC26900187
:103D600098018316980183128C01832EEB30E52E87
:103D7000EC26F600EC26F500EC26F100FB00EC2624
:103D8000F300F20121308312031376020319D12EBE
:103D900075080339FC00FD000310FC0D20307C0782
:103DA000D22E20308400EC268000F207840AFB0B20
:103DB000D32E72087306E830031DE52EE730E726A0
:103DC000FE260038E4300319E530E7269D2E640016
:103DD0000C1EE72E9900080064007A080319FA2ED9
:103DE0000C1CFA2E1010FA0BF62E00340C103C307E
:103DF0008F0010148C1EEC2E1A0808002130760259
:103E00000319502F831603178C1783120313750899
:103E1000FC3903178D000313760803178F00203039
:103E2000840003137D080319282F831603170C142D
:103E30000000000083120E088000840A0C08800035
:103E4000840A8D0A0313FD03F503F10AF10A112F09
:103E50007108FC00203E84000310FC0C7608031758
:103E60008F000313750803178D0003137C080317D5
:103E70008D0703198F0A03170D0803390319502FF3
:103E800083160C140000000083120E088000840AC0
:103E90000C088000840A8D0A0313F10AF10A3B2FF3
:103EA0007508F7007608F800FB010230F40071088D
:103EB0007B02031801347B08203E84002130780205
:103EC0000317831603196E2F8C1783011E30780297
:103ED0008030031977020318B62F702F8C138301DB
:103EE000770803178D0003137808031D852F04300E
:103EF00077020318852F031783168C1F822F8312D6
:103F000084308D0783011E30862F780803178F00B9
:103F100000088E00840A00088C0083160C155530AA
:103F20008D00AA308D008C140000000083018316E0
:103F300003178C1BBE2F8312031364000D1E9D2FCD
:103F40000D12831603170C110C14000000008312CD
:103F5000840300080E06031DB22F840A00080C0615
:103F60000319B62F8301F40B572F00348312031368
:103F70000230FB07F70A0319F80A552F83120313BF
:103F80000D12831603170C11831203170D08033942
:103F9000033C031DB62F03308D028312031304303C
:103FA000FC00073084020000831603170C14000085
:103FB000000000000000000000000008831203174A
:103FC0000E06031DE82F840A00080C060319EF2FC4
:103FD00083120313FC30F7050630FB02B22F831265
:103FE00003178D0A840A83120313FC0BD32FB62FF9
:103FF000FF3FFF3FFF3FFF3FFF3FFF3FFF3FFF3FD1
:084000000F000F000F000F007C
:02400E00313F40
:10420000FF00FF00FF00FF00FF00FF00FF00FF00B6
:10421000FF00FF00FF00FF00FF00FF00FF00FF00A6
:10422000FF00FF00FF00FF00FF00FF00FF00FF0096
:10423000FF00FF00FF00FF00FF00FF00FF00FF0086
:10424000FF00FF00FF00FF00FF00FF00FF00FF0076
:10425000FF00FF00FF00FF00FF00FF00FF00FF0066
:10426000FF00FF00FF00FF00FF00FF00FF00FF0056
:10427000FF00FF00FF00FF00FF00FF00FF00FF0046
:10428000FF00FF00FF00FF00FF00FF00FF00FF0036
:10429000FF00FF00FF00FF00FF00FF00FF00FF0026
:1042A000FF00FF00FF00FF00FF00FF00FF00FF0016
:1042B000FF00FF00FF00FF00FF00FF00FF00FF0006
:1042C000FF00FF00FF00FF00FF00FF00FF00FF00F6
:1042D000FF00FF00FF00FF00FF00FF00FF00FF00E6
:1042E000FF00FF00FF00FF00FF00FF00FF00FF00D6
:1042F000FF00FF00FF00FF00FF00FF00FF00FF00C6
:10430000FF00FF00FF00FF00FF00FF00FF00FF00B5
:10431000FF00FF00FF00FF00FF00FF00FF00FF00A5
:10432000FF00FF00FF00FF00FF00FF00FF00FF0095
:10433000FF00FF00FF00FF00FF00FF00FF00FF0085
:10434000FF00FF00FF00FF00FF00FF00FF00FF0075
:10435000FF00FF00FF00FF00FF00FF00FF00FF0065
:10436000FF00FF00FF00FF00FF00FF00FF00FF0055
:10437000FF00FF00FF00FF00FF00FF00FF00FF0045
:10438000FF00FF00FF00FF00FF00FF00FF00FF0035
:10439000FF00FF00FF00FF00FF00FF00FF00FF0025
:1043A000FF00FF00FF00FF00FF00FF00FF00FF0015
:1043B000FF00FF00FF00FF00FF00FF00FF00FF0005
:1043C000FF00FF00FF00FF00FF00FF00FF00FF00F5
:1043D000FF00FF00FF00FF00FF00FF00FF00FF00E5
:1043E000FF00FF00FF00FF00FF00FF00FF00FF00D5
:1043F000FF00FF00FF00FF00FF00FF00FF00FF00C5
:00000001FF
